BL51 BANKED LINKER/LOCATER V6.02                                                        11/30/2006  10:11:54  PAGE 1


BL51 BANKED LINKER/LOCATER V6.02, INVOKED BY:
C:\PROGRAMFILES\KEIL\C51\BIN\BL51.EXE STARTUP_murphy.obj, main.obj TO debugger_design CODE (0X0000-0XFFFF)


MEMORY MODEL: SMALL WITH FLOATING POINT ARITHMETIC


INPUT MODULES INCLUDED:
  STARTUP_murphy.obj (?C_STARTUP)
  main.obj (MAIN)
  C:\PROGRAMFILES\KEIL\C51\LIB\C51FPS.LIB (?C?FPMUL)
  C:\PROGRAMFILES\KEIL\C51\LIB\C51FPS.LIB (?C?FCAST)
  C:\PROGRAMFILES\KEIL\C51\LIB\C51FPS.LIB (?C?FPGETOPN)
  C:\PROGRAMFILES\KEIL\C51\LIB\C51S.LIB (?C_INIT)
  C:\PROGRAMFILES\KEIL\C51\LIB\C51S.LIB (?C?CLDPTR)
  C:\PROGRAMFILES\KEIL\C51\LIB\C51S.LIB (?C?LNEG)
  C:\PROGRAMFILES\KEIL\C51\LIB\C51S.LIB (?C?ULCMP)
  C:\PROGRAMFILES\KEIL\C51\LIB\C51S.LIB (?C?ULSHR)


LINK MAP OF MODULE:  debugger_design (?C_STARTUP)


            TYPE    BASE      LENGTH    RELOCATION   SEGMENT NAME
            -----------------------------------------------------

            * * * * * * *   D A T A   M E M O R Y   * * * * * * *
            REG     0000H     0008H     ABSOLUTE     "REG BANK 0"
            DATA    0008H     000BH     UNIT         _DATA_GROUP_
            DATA    0013H     0009H     UNIT         ?DT?_GET_FLOAT?MAIN
            DATA    001CH     0004H     UNIT         ?DT?_DLY?MAIN
            DATA    0020H     0003H     UNIT         ?DT?_TX_STR_NO_NL?MAIN
            DATA    0023H     0001H     UNIT         ?DT?MAIN
            IDATA   0024H     0001H     UNIT         ?STACK

            * * * * * * *   C O D E   M E M O R Y   * * * * * * *
            CODE    0000H     0003H     ABSOLUTE     
                    0003H     07FDH                  *** GAP ***
            CODE    0800H     01D9H     UNIT         ?C?LIB_CODE
            CODE    09D9H     00B2H     UNIT         ?PR?_GET_FLOAT?MAIN
            CODE    0A8BH     00ADH     UNIT         ?PR?INIT_ACM?MAIN
            CODE    0B38H     008CH     UNIT         ?C_C51STARTUP
            CODE    0BC4H     0075H     UNIT         ?PR?MAIN?MAIN
            CODE    0C39H     006EH     UNIT         ?PR?_GET_ACM_ADDR?MAIN
            CODE    0CA7H     004FH     UNIT         ?PR?_WR_AQ?MAIN
            CODE    0CF6H     0049H     UNIT         ?PR?_GATE_DRIVER_CTRL?MAIN
            CODE    0D3FH     0044H     UNIT         ?PR?_TXHEX?MAIN
            CODE    0D83H     0036H     UNIT         ?PR?_DLY?MAIN
            CODE    0DB9H     0036H     UNIT         ?PR?_TX_CHAR?MAIN
            CODE    0DEFH     002DH     UNIT         ?PR?_GET_CHAN?MAIN
            CODE    0E1CH     0028H     UNIT         ?PR?_TX_STR?MAIN
            CODE    0E44H     0025H     UNIT         ?PR?_HEX2CHAR?MAIN
            CODE    0E69H     0025H     UNIT         ?CO?MAIN
            CODE    0E8EH     001FH     UNIT         ?PR?_TX_STR_NO_NL?MAIN
            CODE    0EADH     0018H     UNIT         ?PR?INIT_COREAI?MAIN
            CODE    0EC5H     0017H     UNIT         ?PR?_RD_ACM_RAW?MAIN
            CODE    0EDCH     0016H     UNIT         ?PR?RX_CHAR?MAIN
            CODE    0EF2H     0015H     UNIT         ?PR?_DO_VMON_CONVERSION?MAIN
BL51 BANKED LINKER/LOCATER V6.02                                                      11/30/2006  10:11:54  PAGE 2


            CODE    0F07H     0011H     UNIT         ?PR?ADC_CALIBRATE_WAIT?MAIN
            CODE    0F18H     0011H     UNIT         ?PR?ADC_SAMPLE_WAIT?MAIN
            CODE    0F29H     000FH     UNIT         ?PR?ACM_WAIT?MAIN
            CODE    0F38H     000FH     UNIT         ?PR?GET_ADC_VAL?MAIN
            CODE    0F47H     000EH     UNIT         ?PR?_WR_ACM?MAIN
            CODE    0F55H     0009H     UNIT         ?PR?_WR_AQ_AV?MAIN
            CODE    0F5EH     0009H     UNIT         ?PR?_WR_AQ_AC?MAIN
            CODE    0F67H     0009H     UNIT         ?PR?_WR_AQ_AT?MAIN
            CODE    0F70H     0009H     UNIT         ?PR?_WR_AQ_AG?MAIN
            CODE    0F79H     0005H     UNIT         ?PR?_RD_VOLTAGE?MAIN
            CODE    0F7EH     0005H     UNIT         ?PR?_PRESCALED_VMON_CONVERSION?MAIN
            CODE    0F83H     0005H     UNIT         ?PR?_NON_PRESCALED_VMON_CONVERSION?MAIN
            CODE    0F88H     0004H     UNIT         ?C_INITSEG



OVERLAY MAP OF MODULE:   debugger_design (?C_STARTUP)


SEGMENT                                           DATA_GROUP 
  +--> CALLED SEGMENT                           START    LENGTH
---------------------------------------------------------------
?C_C51STARTUP                                   -----    -----
  +--> ?PR?MAIN?MAIN
  +--> ?C_INITSEG

?PR?MAIN?MAIN                                   0008H    0004H
  +--> ?PR?INIT_COREAI?MAIN
  +--> ?CO?MAIN
  +--> ?PR?_TX_STR?MAIN
  +--> ?PR?RX_CHAR?MAIN
  +--> ?PR?_GET_CHAN?MAIN
  +--> ?PR?_PRESCALED_VMON_CONVERSION?MAIN
  +--> ?PR?GET_ADC_VAL?MAIN
  +--> ?PR?_TX_CHAR?MAIN
  +--> ?PR?_TXHEX?MAIN

?PR?INIT_COREAI?MAIN                            -----    -----
  +--> ?PR?ACM_WAIT?MAIN
  +--> ?PR?INIT_ACM?MAIN

?PR?INIT_ACM?MAIN                               -----    -----
  +--> ?PR?_WR_AQ?MAIN
  +--> ?PR?ACM_WAIT?MAIN

?PR?_WR_AQ?MAIN                                 000CH    0005H
  +--> ?PR?_WR_AQ_AV?MAIN
  +--> ?PR?_WR_AQ_AC?MAIN
  +--> ?PR?_WR_AQ_AG?MAIN
  +--> ?PR?_WR_AQ_AT?MAIN

?PR?_WR_AQ_AV?MAIN                              -----    -----
  +--> ?PR?_WR_ACM?MAIN

?PR?_WR_ACM?MAIN                                -----    -----
  +--> ?PR?_GET_ACM_ADDR?MAIN

BL51 BANKED LINKER/LOCATER V6.02                                                      11/30/2006  10:11:54  PAGE 3


?PR?_GET_ACM_ADDR?MAIN                          -----    -----
  +--> ?PR?ACM_WAIT?MAIN

?PR?_WR_AQ_AC?MAIN                              -----    -----
  +--> ?PR?_WR_ACM?MAIN

?PR?_WR_AQ_AG?MAIN                              -----    -----
  +--> ?PR?_WR_ACM?MAIN

?PR?_WR_AQ_AT?MAIN                              -----    -----
  +--> ?PR?_WR_ACM?MAIN

?PR?_TX_STR?MAIN                                000CH    0003H
  +--> ?PR?_TX_CHAR?MAIN

?PR?_PRESCALED_VMON_CONVERSION?MAIN             -----    -----
  +--> ?PR?_DO_VMON_CONVERSION?MAIN

?PR?_DO_VMON_CONVERSION?MAIN                    -----    -----
  +--> ?PR?ADC_CALIBRATE_WAIT?MAIN
  +--> ?PR?ADC_SAMPLE_WAIT?MAIN

?PR?_TXHEX?MAIN                                 000CH    0007H
  +--> ?PR?_HEX2CHAR?MAIN
  +--> ?PR?_TX_CHAR?MAIN



SYMBOL TABLE OF MODULE:  debugger_design (?C_STARTUP)

  VALUE           TYPE          NAME
  ----------------------------------

  -------         MODULE        ?C_STARTUP
  C:0B38H         SEGMENT       ?C_C51STARTUP
  I:0024H         SEGMENT       ?STACK
  C:0000H         PUBLIC        ?C_STARTUP
  D:00E0H         SYMBOL        ACC
  D:00F0H         SYMBOL        B
  D:0083H         SYMBOL        DPH
  D:0082H         SYMBOL        DPL
  N:0000H         SYMBOL        IBPSTACK
  N:0100H         SYMBOL        IBPSTACKTOP
  N:0080H         SYMBOL        IDATALEN
  C:0B3BH         SYMBOL        IDATALOOP
  N:0000H         SYMBOL        PBPSTACK
  N:0000H         SYMBOL        PBPSTACKTOP
  N:0000H         SYMBOL        PDATALEN
  N:0000H         SYMBOL        PDATASTART
  N:0000H         SYMBOL        PPAGE
  N:0000H         SYMBOL        PPAGEENABLE
  D:00A0H         SYMBOL        PPAGE_SFR
  D:0081H         SYMBOL        SP
  C:0B38H         SYMBOL        STARTUP1
  N:0000H         SYMBOL        XBPSTACK
  N:0000H         SYMBOL        XBPSTACKTOP
  N:0000H         SYMBOL        XDATALEN
BL51 BANKED LINKER/LOCATER V6.02                                                      11/30/2006  10:11:54  PAGE 4


  N:0000H         SYMBOL        XDATASTART
  C:0000H         LINE#         92
  C:0B38H         LINE#         99
  C:0B3AH         LINE#         100
  C:0B3BH         LINE#         101
  C:0B3CH         LINE#         102
  C:0B3EH         LINE#         151
  C:0B41H         LINE#         155
  -------         ENDMOD        ?C_STARTUP

  -------         MODULE        MAIN
  C:0000H         SYMBOL        _ICE_DUMMY_
  C:0F7EH         PUBLIC        _prescaled_vmon_conversion
  C:0EADH         PUBLIC        init_coreai
  D:0023H         SYMBOL        rtccnt
  C:0EC5H         PUBLIC        _rd_acm_raw
  C:0E44H         PUBLIC        _hex2char
  C:0CA7H         PUBLIC        _wr_aq
  D:009DH         PUBLIC        XRB1
  C:0E8EH         PUBLIC        _tx_str_no_nl
  D:009AH         PUBLIC        XWB1
  C:0EF2H         PUBLIC        _do_vmon_conversion
  C:0BC4H         PUBLIC        main
  C:0E1CH         PUBLIC        _tx_str
  C:0F18H         PUBLIC        adc_sample_wait
  C:0CF6H         PUBLIC        _gate_driver_ctrl
  C:0F79H         PUBLIC        _rd_voltage
  C:0D3FH         PUBLIC        _txhex
  C:0F83H         PUBLIC        _non_prescaled_vmon_conversion
  C:09D9H         PUBLIC        _get_float
  C:0DEFH         PUBLIC        _get_chan
  C:0F5EH         PUBLIC        _wr_aq_ac
  C:0F70H         PUBLIC        _wr_aq_ag
  C:0A8BH         PUBLIC        init_acm
  C:0F29H         PUBLIC        acm_wait
  C:0D83H         PUBLIC        _dly
  C:0F07H         PUBLIC        adc_calibrate_wait
  C:0C40H         PUBLIC        _get_acm_addr
  C:0F67H         PUBLIC        _wr_aq_at
  C:0F55H         PUBLIC        _wr_aq_av
  C:0EDCH         PUBLIC        rx_char
  C:0DBFH         PUBLIC        _tx_char
  C:0F38H         PUBLIC        get_adc_val
  C:0F47H         PUBLIC        _wr_acm
  -------         PROC          _DLY
  D:0004H         SYMBOL        d
  -------         DO            
  D:001CH         SYMBOL        dcnt
  -------         ENDDO         
  C:0D83H         LINE#         70
  C:0D83H         LINE#         72
  C:0D8BH         LINE#         73
  C:0D9EH         LINE#         74
  C:0DB8H         LINE#         75
  -------         ENDPROC       _DLY
  -------         PROC          _HEX2CHAR
  D:0007H         SYMBOL        h
BL51 BANKED LINKER/LOCATER V6.02                                                      11/30/2006  10:11:54  PAGE 5


  -------         DO            
  D:0006H         SYMBOL        c
  -------         ENDDO         
  C:0E44H         LINE#         78
  C:0E44H         LINE#         80
  C:0E46H         LINE#         81
  C:0E52H         LINE#         83
  C:0E56H         LINE#         84
  C:0E56H         LINE#         85
  C:0E62H         LINE#         86
  C:0E66H         LINE#         87
  C:0E66H         LINE#         88
  C:0E68H         LINE#         89
  -------         ENDPROC       _HEX2CHAR
  -------         PROC          ACM_WAIT
  -------         DO            
  D:0007H         SYMBOL        busy
  -------         ENDDO         
  C:0F29H         LINE#         297
  C:0F29H         LINE#         301
  C:0F2BH         LINE#         302
  C:0F2EH         LINE#         303
  C:0F35H         LINE#         304
  C:0F37H         LINE#         305
  -------         ENDPROC       ACM_WAIT
  -------         PROC          _GET_CHAN
  D:0007H         SYMBOL        t
  D:0005H         SYMBOL        n
  -------         DO            
  D:0006H         SYMBOL        chan
  -------         ENDDO         
  C:0DEFH         LINE#         308
  C:0DEFH         LINE#         310
  C:0DFAH         LINE#         311
  C:0E03H         LINE#         312
  C:0E0DH         LINE#         313
  C:0E17H         LINE#         314
  C:0E19H         LINE#         315
  C:0E19H         LINE#         316
  C:0E1BH         LINE#         317
  -------         ENDPROC       _GET_CHAN
  -------         PROC          L?0106
  -------         ENDPROC       L?0106
  -------         PROC          _GET_ACM_ADDR
  D:0007H         SYMBOL        t
  D:0005H         SYMBOL        n
  -------         DO            
  D:0006H         SYMBOL        addr
  -------         ENDDO         
  C:0C40H         LINE#         321
  C:0C40H         LINE#         323
  C:0C65H         LINE#         324
  C:0C6EH         LINE#         325
  C:0C78H         LINE#         326
  C:0C82H         LINE#         327
  C:0C8CH         LINE#         328
  C:0C92H         LINE#         329
BL51 BANKED LINKER/LOCATER V6.02                                                      11/30/2006  10:11:54  PAGE 6


  C:0C98H         LINE#         330
  C:0C9EH         LINE#         331
  C:0CA2H         LINE#         332
  C:0CA4H         LINE#         333
  C:0CA4H         LINE#         334
  C:0CA6H         LINE#         335
  -------         ENDPROC       _GET_ACM_ADDR
  -------         PROC          _WR_ACM
  D:0006H         SYMBOL        t
  D:0005H         SYMBOL        n
  D:0003H         SYMBOL        d
  C:0F47H         LINE#         338
  C:0F47H         LINE#         340
  C:0F47H         LINE#         342
  C:0F4FH         LINE#         344
  C:0F54H         LINE#         345
  -------         ENDPROC       _WR_ACM
  -------         PROC          _RD_ACM_RAW
  D:0006H         SYMBOL        t
  D:0005H         SYMBOL        n
  -------         DO            
  D:0007H         SYMBOL        rdhold
  -------         ENDDO         
  C:0EC5H         LINE#         349
  C:0EC5H         LINE#         352
  C:0EC5H         LINE#         354
  C:0ECDH         LINE#         356
  C:0ED3H         LINE#         358
  C:0ED6H         LINE#         360
  C:0EDBH         LINE#         361
  C:0EDBH         LINE#         362
  -------         ENDPROC       _RD_ACM_RAW
  -------         PROC          _RD_VOLTAGE
  D:0001H         SYMBOL        addr
  -------         DO            
  D:0007H         SYMBOL        rdhold
  -------         ENDDO         
  C:0F79H         LINE#         366
  C:0F79H         LINE#         368
  C:0F7DH         LINE#         369
  C:0F7DH         LINE#         370
  -------         ENDPROC       _RD_VOLTAGE
  -------         PROC          _WR_AQ_AV
  D:0005H         SYMBOL        n
  D:0003H         SYMBOL        d
  C:0F55H         LINE#         374
  C:0F59H         LINE#         375
  -------         ENDPROC       _WR_AQ_AV
  -------         PROC          _WR_AQ_AC
  D:0005H         SYMBOL        n
  D:0003H         SYMBOL        d
  C:0F5EH         LINE#         378
  C:0F62H         LINE#         379
  -------         ENDPROC       _WR_AQ_AC
  -------         PROC          _WR_AQ_AT
  D:0005H         SYMBOL        n
  D:0003H         SYMBOL        d
BL51 BANKED LINKER/LOCATER V6.02                                                      11/30/2006  10:11:54  PAGE 7


  C:0F67H         LINE#         382
  C:0F6BH         LINE#         383
  -------         ENDPROC       _WR_AQ_AT
  -------         PROC          _WR_AQ_AG
  D:0005H         SYMBOL        n
  D:0003H         SYMBOL        d
  C:0F70H         LINE#         386
  C:0F74H         LINE#         387
  -------         ENDPROC       _WR_AQ_AG
  -------         PROC          _WR_AQ
  D:0002H         SYMBOL        n
  D:000DH         SYMBOL        d
  C:0CA7H         LINE#         391
  C:0CA9H         LINE#         392
  C:0CAEH         LINE#         393
  C:0CC6H         LINE#         394
  C:0CDEH         LINE#         395
  -------         ENDPROC       _WR_AQ
  -------         PROC          INIT_ACM
  C:0A8BH         LINE#         399
  C:0A8BH         LINE#         401
  C:0A9CH         LINE#         402
  C:0AADH         LINE#         403
  C:0ABEH         LINE#         404
  C:0ACFH         LINE#         405
  C:0AE0H         LINE#         406
  C:0AF1H         LINE#         407
  C:0B02H         LINE#         408
  C:0B13H         LINE#         409
  C:0B24H         LINE#         410
  C:0B35H         LINE#         411
  -------         ENDPROC       INIT_ACM
  -------         PROC          ADC_CALIBRATE_WAIT
  -------         DO            
  D:0007H         SYMBOL        busy
  -------         ENDDO         
  C:0F07H         LINE#         415
  C:0F07H         LINE#         417
  C:0F07H         LINE#         418
  C:0F09H         LINE#         419
  C:0F0CH         LINE#         420
  C:0F10H         LINE#         421
  C:0F15H         LINE#         422
  C:0F17H         LINE#         423
  -------         ENDPROC       ADC_CALIBRATE_WAIT
  -------         PROC          ADC_SAMPLE_WAIT
  -------         DO            
  D:0007H         SYMBOL        busy
  -------         ENDDO         
  C:0F18H         LINE#         426
  C:0F18H         LINE#         428
  C:0F18H         LINE#         429
  C:0F1AH         LINE#         430
  C:0F1DH         LINE#         431
  C:0F21H         LINE#         432
  C:0F26H         LINE#         433
  C:0F28H         LINE#         434
BL51 BANKED LINKER/LOCATER V6.02                                                      11/30/2006  10:11:54  PAGE 8


  -------         ENDPROC       ADC_SAMPLE_WAIT
  -------         PROC          _DO_VMON_CONVERSION
  D:0006H         SYMBOL        n
  D:0005H         SYMBOL        stc
  C:0EF2H         LINE#         438
  C:0EF4H         LINE#         439
  C:0EF7H         LINE#         440
  C:0EFAH         LINE#         443
  C:0EFFH         LINE#         444
  C:0F04H         LINE#         445
  -------         ENDPROC       _DO_VMON_CONVERSION
  -------         PROC          _PRESCALED_VMON_CONVERSION
  D:0007H         SYMBOL        n
  C:0F7EH         LINE#         450
  C:0F7EH         LINE#         452
  -------         ENDPROC       _PRESCALED_VMON_CONVERSION
  -------         PROC          _NON_PRESCALED_VMON_CONVERSION
  D:0007H         SYMBOL        n
  C:0F83H         LINE#         457
  C:0F83H         LINE#         459
  -------         ENDPROC       _NON_PRESCALED_VMON_CONVERSION
  -------         PROC          GET_ADC_VAL
  -------         DO            
  D:0004H         SYMBOL        result
  -------         ENDDO         
  C:0F38H         LINE#         464
  C:0F38H         LINE#         466
  C:0F3DH         LINE#         467
  C:0F42H         LINE#         468
  C:0F46H         LINE#         469
  -------         ENDPROC       GET_ADC_VAL
  -------         PROC          _GET_FLOAT
  D:0007H         SYMBOL        r
  D:0014H         SYMBOL        d
  -------         DO            
  D:0018H         SYMBOL        f
  -------         ENDDO         
  C:09D9H         LINE#         473
  C:09D9H         LINE#         475
  C:0A04H         LINE#         477
  C:0A0FH         LINE#         478
  C:0A1AH         LINE#         479
  C:0A28H         LINE#         480
  C:0A33H         LINE#         481
  C:0A41H         LINE#         482
  C:0A4CH         LINE#         483
  C:0A5AH         LINE#         484
  C:0A5CH         LINE#         485
  C:0A67H         LINE#         486
  C:0A73H         LINE#         487
  C:0A73H         LINE#         488
  C:0A8AH         LINE#         489
  -------         ENDPROC       _GET_FLOAT
  -------         PROC          INIT_COREAI
  C:0EADH         LINE#         492
  C:0EADH         LINE#         494
  C:0EB3H         LINE#         495
BL51 BANKED LINKER/LOCATER V6.02                                                      11/30/2006  10:11:54  PAGE 9


  C:0EB6H         LINE#         497
  C:0EB9H         LINE#         498
  C:0EBFH         LINE#         499
  C:0EC2H         LINE#         500
  -------         ENDPROC       INIT_COREAI
  -------         PROC          _GATE_DRIVER_CTRL
  D:0006H         SYMBOL        ag
  D:0005H         SYMBOL        o
  -------         DO            
  D:0002H         SYMBOL        gdstate
  D:0004H         SYMBOL        gdmask
  D:0001H         SYMBOL        gdon
  -------         ENDDO         
  C:0CF6H         LINE#         504
  C:0CF8H         LINE#         508
  C:0CFBH         LINE#         509
  C:0CFEH         LINE#         510
  C:0D02H         LINE#         511
  C:0D17H         LINE#         513
  C:0D1CH         LINE#         514
  C:0D20H         LINE#         516
  C:0D23H         LINE#         517
  C:0D2BH         LINE#         519
  C:0D35H         LINE#         520
  C:0D37H         LINE#         521
  C:0D3EH         LINE#         522
  -------         ENDPROC       _GATE_DRIVER_CTRL
  -------         PROC          RX_CHAR
  -------         DO            
  D:0006H         SYMBOL        ret
  D:0005H         SYMBOL        rxrdy
  -------         ENDDO         
  C:0EDCH         LINE#         55
  C:0EDCH         LINE#         58
  C:0EDEH         LINE#         59
  C:0EE4H         LINE#         60
  C:0EE6H         LINE#         61
  C:0EEBH         LINE#         62
  C:0EEDH         LINE#         63
  C:0EF1H         LINE#         64
  C:0EF1H         LINE#         65
  C:0EF1H         LINE#         66
  -------         ENDPROC       RX_CHAR
  -------         PROC          L?0107
  -------         ENDPROC       L?0107
  -------         PROC          _TX_CHAR
  D:0007H         SYMBOL        c
  -------         DO            
  D:0006H         SYMBOL        ret
  D:0003H         SYMBOL        txrdy
  D:0004H         SYMBOL        i
  -------         ENDDO         
  C:0DBFH         LINE#         69
  C:0DBFH         LINE#         73
  C:0DC1H         LINE#         74
  C:0DC3H         LINE#         75
  C:0DCAH         LINE#         78
BL51 BANKED LINKER/LOCATER V6.02                                                      11/30/2006  10:11:54  PAGE 10


  C:0DCDH         LINE#         79
  C:0DD4H         LINE#         81
  C:0DDBH         LINE#         82
  C:0DDBH         LINE#         83
  C:0DDBH         LINE#         84
  C:0DE0H         LINE#         85
  C:0DE0H         LINE#         86
  C:0DE2H         LINE#         87
  C:0DE5H         LINE#         88
  C:0DEAH         LINE#         89
  C:0DECH         LINE#         91
  C:0DECH         LINE#         92
  C:0DEEH         LINE#         93
  -------         ENDPROC       _TX_CHAR
  -------         PROC          _TX_STR
  D:000CH         SYMBOL        s
  C:0E1CH         LINE#         98
  C:0E22H         LINE#         99
  C:0E2DH         LINE#         100
  C:0E3AH         LINE#         101
  C:0E3FH         LINE#         102
  -------         ENDPROC       _TX_STR
  -------         PROC          _TX_STR_NO_NL
  D:0020H         SYMBOL        s
  C:0E8EH         LINE#         106
  C:0E94H         LINE#         107
  C:0E9FH         LINE#         108
  C:0EACH         LINE#         109
  -------         ENDPROC       _TX_STR_NO_NL
  -------         PROC          _TXHEX
  D:000CH         SYMBOL        d
  D:0010H         SYMBOL        w
  -------         DO            
  D:0011H         SYMBOL        i
  -------         ENDDO         
  C:0D3FH         LINE#         113
  C:0D47H         LINE#         115
  C:0D57H         LINE#         116
  C:0D82H         LINE#         117
  -------         ENDPROC       _TXHEX
  -------         PROC          MAIN
  -------         DO            
  D:0008H         SYMBOL        ctmp
  D:000AH         SYMBOL        sample16
  -------         ENDDO         
  C:0BC4H         LINE#         23
  C:0BC4H         LINE#         28
  C:0BCAH         LINE#         29
  C:0BD0H         LINE#         32
  C:0BD6H         LINE#         35
  C:0BD9H         LINE#         38
  C:0BE2H         LINE#         41
  C:0BE2H         LINE#         43
  C:0BE9H         LINE#         44
  C:0BF3H         LINE#         46
  C:0BFDH         LINE#         47
  C:0C04H         LINE#         49
BL51 BANKED LINKER/LOCATER V6.02                                                      11/30/2006  10:11:54  PAGE 11


  C:0C0DH         LINE#         50
  C:0C12H         LINE#         51
  C:0C1BH         LINE#         52
  C:0C28H         LINE#         54
  C:0C32H         LINE#         56
  C:0C37H         LINE#         58
  C:0C37H         LINE#         59
  -------         ENDPROC       MAIN
  -------         ENDMOD        MAIN

  -------         MODULE        ?C?FPMUL
  C:0800H         PUBLIC        ?C?FPMUL
  -------         ENDMOD        ?C?FPMUL

  -------         MODULE        ?C?FCAST
  C:0910H         PUBLIC        ?C?FCASTC
  C:090BH         PUBLIC        ?C?FCASTI
  C:0906H         PUBLIC        ?C?FCASTL
  -------         ENDMOD        ?C?FCAST

  -------         MODULE        ?C?CLDPTR
  C:098EH         PUBLIC        ?C?CLDPTR
  -------         ENDMOD        ?C?CLDPTR

  -------         MODULE        ?C?LNEG
  C:09A7H         PUBLIC        ?C?LNEG
  -------         ENDMOD        ?C?LNEG

  -------         MODULE        ?C?ULCMP
  C:09B5H         PUBLIC        ?C?ULCMP
  -------         ENDMOD        ?C?ULCMP

  -------         MODULE        ?C?ULSHR
  C:09C6H         PUBLIC        ?C?ULSHR
  -------         ENDMOD        ?C?ULSHR

*** WARNING L16: UNCALLED SEGMENT, IGNORED FOR OVERLAY PROCESS
    SEGMENT: ?PR?_DLY?MAIN

*** WARNING L16: UNCALLED SEGMENT, IGNORED FOR OVERLAY PROCESS
    SEGMENT: ?PR?_RD_ACM_RAW?MAIN

*** WARNING L16: UNCALLED SEGMENT, IGNORED FOR OVERLAY PROCESS
    SEGMENT: ?PR?_RD_VOLTAGE?MAIN

*** WARNING L16: UNCALLED SEGMENT, IGNORED FOR OVERLAY PROCESS
    SEGMENT: ?PR?_NON_PRESCALED_VMON_CONVERSION?MAIN

*** WARNING L16: UNCALLED SEGMENT, IGNORED FOR OVERLAY PROCESS
    SEGMENT: ?PR?_GET_FLOAT?MAIN

*** WARNING L16: UNCALLED SEGMENT, IGNORED FOR OVERLAY PROCESS
    SEGMENT: ?PR?_GATE_DRIVER_CTRL?MAIN

*** WARNING L16: UNCALLED SEGMENT, IGNORED FOR OVERLAY PROCESS
    SEGMENT: ?PR?_TX_STR_NO_NL?MAIN

BL51 BANKED LINKER/LOCATER V6.02                                                      11/30/2006  10:11:54  PAGE 12


******************************************************************************
* RESTRICTED VERSION WITH 0800H BYTE CODE SIZE LIMIT; USED: 0535H BYTE (65%) *
******************************************************************************

Program Size: data=37.0 xdata=0 code=1935
LINK/LOCATE RUN COMPLETE.  7 WARNING(S),  0 ERROR(S)
